:100000002BC009C012C01BC01BC01BC01BC01BC023
:1000100020C020C020C00FB60F9251E0F52EFAD0BC
:1000200050E45ABF0F900FBE18950FB60F9252E0D2
:10003000F52EF0D050E85ABF0F900FBE18951895C6
:100040001895189518950FB60F9269D00F900FBE9E
:1000500018951895189518950FED0DBF00E008BB81
:1000600000E102BB00E007BB02E101BB442711270E
:10007000949A0CE04A95F1F71A95E1F70A95D1F7B1
:1000800094980CE04A95F1F71A95E1F70A95D1F7A3
:10009000949A0CE04A95F1F71A95E1F70A95D1F791
:1000A00094980CE04A95F1F71A95E1F70A95D1F783
:1000B000949A0AE005BF00E00BBF00E00ABF00E031
:1000C00009BF0AEC08BF00E003BF00E00FBD00E07D
:1000D0000EBD00E00DBD00E00CBD00E00BBD00E07A
:1000E0000ABD00E001BD08E90AB904E0859909E00C
:1000F00009B900E008B9B0E0A8E5D0E0C0E6F0E05A
:10010000E0E000E00993C03EE9F700E00093600002
:1001100000E00093610000E00BBF7894FFCF5CB17A
:10012000573429F450EC5ABF60EC6BBF72C05534A1
:1001300029F460E06BBF3FEFBAD06BC0563511F4C5
:10014000C0D067C0533521F436B3B1D0B4D061C04C
:10015000503371F460E06BBF60E0E62E6BE0A62EDA
:100160006BE2B62E67E0C62E69E8D62EA4D051C049
:10017000513371F460E06BBF61E0E62E65E0A62EBE
:1001800064E8B62E63E0C62E65ECD62E94D041C04E
:10019000523371F460E06BBF62E0E62E62E0A62E9F
:1001A00060EBB62E61E0C62E62EED62E84D031C052
:1001B000533371F460E06BBF63E0E62E61E0A62E7E
:1001C0006FEBB62E61E0C62E62E4D62E74D021C04D
:1001D000543371F460E06BBF64E0E62E61E0A62E5C
:1001E00067E4B62E60E0C62E61EFD62E64D011C053
:1001F000553371F460E06BBF65E0E62E60E0A62E3B
:100200006EECB62E60E0C62E61EAD62E54D001C048
:1002100055D0089550E05EBD50E05DBD50E05CBD3E
:10022000ABBCBABC50E458BF59E05EBD88249924E9
:1002300098E058B756FFFDCF8C98CBBCDABC50E4A1
:1002400058BF80B3669576956F7782FD60687F773B
:1002500083FD70688C9A9A9561F7862E972E50E0F0
:100260005EBDABBCBABC50E458BF5F2D513061F4E9
:10027000582D52955F705068352F19D0582D5F70EA
:100280005069352F14D00EC0523061F4592D52955B
:100290005F70506A352F0BD0592D5F70506B352F22
:1002A00006D000C0829BFECF839BFECF08955D9B4E
:1002B000FECF3CB908953DE0FADF08953FE3F7DF54
:1002C000089531E4F4DF36E7F2DF32E7F0DF30E2C1
:1002D000EEDF32E5ECDF33E5EADF32E3E8DF33E39C
:1002E000E6DF32E3E4DF30E2E2DF36E5E0DF31E3B0
:1002F000DEDF3EE2DCDF30E3DADF31E3D8DF30E2BD
:10030000D6DF2E2D203061F430E2D1DF34E3CFDFB1
:1003100038E3CDDF30E3CBDF30E3C9DFCCDF51C0E2
:10032000213061F430E2C3DF39E3C1DF36E3BFDF00
:1003300030E3BDDF30E3BBDFBEDF43C0223061F41A
:1003400031E3B5DF39E3B3DF32E3B1DF30E3AFDF11
:1003500030E3ADDFB0DF35C0233061F432E3A7DF37
:1003600038E3A5DF38E3A3DF30E3A1DF30E39FDF2D
:10037000A2DF27C0243061F433E399DF38E397DF4D
:1003800034E395DF30E393DF30E391DF94DF19C08E
:10039000253061F435E38BDF37E389DF36E387DF30
:1003A00030E385DF30E383DF86DF0BC03FE37FDFB1
:1003B0003FE37DDF3FE37BDF3FE379DF3FE377DF51
:0403C0007ADF089543
:00000001FF
